:020000040000FA
:1000000083168E18C02883120130162086018701BE
:1000100083168E148F30810006309F00D03085000B
:10002000003086007F30870083127D28A200FF30D9
:10003000A100FF30A00064000000A00B1C28A10B51
:100040001928A20B172808000739051E3028820737
:10005000033406340C340934033406340C340934C4
:100060008207013403340234063404340C34083477
:1000700009340739051E4528820730346034C034FE
:10008000903430346034C0349034820710343034CB
:10009000203460344034C034803490342314871CBE
:1000A0005828A40324082420A80027048600080058
:1000B000A40A24082420A800270486000800A3140A
:1000C000871D6928A50325083920A7002804860074
:1000D0000800A50A25083920A70028048600080082
:1000E0002315871E7828A6032608242085000800EB
:1000F000A60A2608242085000800A3018701A7017D
:10010000A80185016400071BA72823188A2807185F
:100110004E2090288316071007148312071C231003
:10012000A318952807195F209B2883160711071528
:100130008312071DA3102319A028071A70208228F4
:100140008316071207168312071E231182288316AF
:10015000DF308500FF3086008312071FB82887171D
:10016000043016208713071FB82804301620AD2846
:1001700087018316D03085000030860083128228E4
:100180007F30870083121430162087170230162024
:100190008713043016208717023016208713043087
:1001A000162087170230162087130830162087176D
:1001B00006301620871304301620871706301620C5
:1001C000871304301620871706301620871308304F
:1001D0001620871702301620871304301620871741
:1001E000023016208713043016208717023016209D
:0401F0008713C32886
:084000000000010000000000B7
:02400E003E3F33
:00000001FF
